:100000000C94C9000C94AC0B0C94E6000C94E60024
:100010000C94E6000C94E6000C94E6000C94E600C8
:100020000C94E6000C94E6000C94E6000C9423017A
:100030000C94E6000C94E6000C94E6000C94FF008F
:100040000C94E6000C94E6000C94E6000C94710904
:100050000C94890A0C94E6000C94E6000C94E600DB
:100060000C94E6000C94E6000C94E6000C94E60078
:10007000C102C702EE02FC02080310032103290398
:100080003A0353036F038503BD032A0460046C0421
:100090007C048604980473058005B4052020202084
:1000A00020434D746563202020202020726F626FF2
:1000B000437261776C65722076312E3120202020CA
:1000C0002020202020202020202020200020202050
:1000D00020206D6F646520313A2020202020466F5B
:1000E0006C6C6F772077616C6C20617420206120CC
:1000F00064697374616E636528316D292000202066
:100100002020206D6F646520323A2020202020447A
:100110007269766520616E6420766F6964202020A4
:1001200020616E792077616C6C7320202020002084
:10013000202020206D6F646520333A202020204D40
:100140006561737572652064697374616E6365209F
:10015000202020666F7277617264202020202000AA
:10016000202020206D6F64652052463A20202020F8
:10017000205246206163746976656420616E642054
:1001800077616974696E6720666F7220636F6D2E88
:10019000000011241FBECFEFD4E0DEBFCDBF14E0BE
:1001A000A0E0B1E0EAE4F8E102C005900D92AA32C5
:1001B000B107D9F714E0AAE2B4E001C01D92A53658
:1001C000B107E1F70E9418070C94240C0C9400006E
:1001D00082E08EBD8FEB8DBD8FEF8CBD8EEE83BD2B
:1001E00089B7846889BF84B3876084BB8AB38F7002
:1001F0008ABB8BB3806F8BBB10922F0408951F9224
:100200000F920FB60F9211248F9380912C048F5F61
:1002100080932C04823050F010922A0485B38760BA
:1002200085BB87B5826087BD10922C0481E08093E6
:1002300030048FEB8DBD8FEF8CBD8F910F900FBE73
:100240000F901F9018951F920F920FB60F921124C6
:100250002F938F939F9390912A0480910304981772
:1002600018F0A99821E002C0000020E08091040469
:10027000981710F0A89802C0000020E080910504B3
:10028000981720F0AA98222319F406C0000004C091
:1002900087B58D7F87BD05C09F5F90932A040000BE
:1002A00000008EEE83BD9F918F912F910F900FBE16
:1002B0000F901F9018951F93182F80E00E94A80799
:1002C00081E3189FC001112484569F4F0E942D087E
:1002D00088EC80932E0410933B041F910895109294
:1002E0003B0487E780930404809305048CE88093A3
:1002F00003040E94BB0908951F93CF93DF93EC0181
:10030000162F413011F480E007C0423011F480E133
:1003100003C0433019F480E20E94D3071123B9F5DA
:100320008DE7C130D807C8F58EE3C138D80718F07B
:1003300081E191E0CAC08FE1C134D80718F082E2B0
:1003400091E0C3C08FE0C13AD80718F083E391E091
:10035000BCC087E0C13DD80718F084E491E0B5C087
:1003600083E0C93ED80718F085E591E0AEC081E092
:10037000C53FD80718F086E691E0A7C0C536D1057D
:1003800018F087E791E0A1C088E891E09EC01130A5
:10039000D1F58DE7C130D80718F080E091E095C025
:1003A0008EE3C138D80718F089E991E08EC08FE15B
:1003B000C134D80718F08AEA91E087C08FE0C13ACB
:1003C000D80718F08BEB91E080C087E0C13DD807DB
:1003D00018F08CEC91E079C083E0C93ED80718F0A2
:1003E0008DED91E072C081E0C53FD80718F08EEE28
:1003F00091E06BC0C536D10518F08FEF91E065C074
:1004000080E192E062C0123071F589E1C130D80715
:1004100018F081E292E059C08CE0C138D80718F09A
:1004200082E392E052C086E0C134D80718F083E43A
:1004300092E04BC083E0C132D80718F084E592E027
:1004400044C081E0C139D80718F085E692E03DC08C
:10045000C93CD10518F086E792E037C06F9798F154
:1004600087E892E032C0133091F589E1C130D807B6
:1004700018F089EA92E029C08CE0C138D80718F05A
:100480008AEB92E022C086E0C134D80718F08BECEA
:1004900092E01BC083E0C132D80718F08CED92E0E7
:1004A00014C081E0C139D80718F08DEE92E00DC07C
:1004B000C93CD10518F08EEF92E007C06F9718F095
:1004C0008FE093E002C088E992E00E943B08DF9150
:1004D000CF911F9108950F931F930E946D09882358
:1004E00061F00E9464098C0183E10E94D307C80176
:1004F0000E943B08C8010E94130A0E94C30983306E
:1005000061F0843018F4823099F405C0843059F0D9
:10051000853071F40BC081E001C082E00E945B0174
:100520000E94BF0905C00E946F0102C00E946909B4
:100530001F910F9108951F9380913C04882311F01F
:100540000E946B0280913B04813009F01EC38091B0
:100550002D048F5F80932D0490912E04891708F449
:1005600014C380912F04E82FF0E0E631F10508F084
:100570000AC3E85CFF4FEE0FFF1F0590F491E02DDA
:1005800009940E94DF0781E00E94A807A5C18FE7B8
:1005900080930404809305040E948C0B84E0809374
:1005A0002E040E94A70B882309F4EDC20E94A00B21
:1005B000909332048093310427E18037920738F416
:1005C00042E060E080E090E00E947C01AFC142E048
:1005D00060E0805797410E947C01D5C280E00E9474
:1005E000D30781E393E00E943B088CE680930404E8
:1005F0008093050488E27DC187E78093040480939B
:10060000050481E080932E041092420484E0B9C274
:100610008EEA8093030484E180932E0485E0B1C2C6
:100620000E948C0B84E080932E040E94A70B8823E9
:1006300009F4A9C20E94A00B909338048093370458
:1006400075C187E68093030488E280932E0487E0D7
:1006500098C20E948C0B84E080932E040E94A70B0A
:10066000882309F490C20E94A00B90933A048093CF
:1006700039045CC18CE880930304209137043091E5
:1006800038048091390490913A048217930718F442
:1006900010923F0403C081E080933F0482E3809383
:1006A0002E0489E06EC20E948C0B84E080932E049D
:1006B0000E94A70B882309F466C280E00E94D3073A
:1006C00082E493E00E943B080E94A00B90933604C2
:1006D00080933504909334048093330427C1809130
:1006E0003F04882329F486E88093040488E606C042
:1006F000813049F488E68093040486E880930504F9
:1007000087E080932E048BE03CC20E948C0B84E037
:1007100080932E0487E780930404809305040E944D
:10072000A70B882309F42FC20E94A00B90933204D8
:10073000809331042091350430913604281739070D
:1007400070F480E00E94D30783E593E00E943B08A9
:1007500081E080932E0480912F048F5F03C08091ED
:100760002F04815080932F048091310490913204A2
:10077000909336048093350406C20E948C0B84E06B
:1007800080932E040E94A70B882309F4FCC10E94C9
:10079000A00B9C01909332048093310447E1813790
:1007A000940728F042E060E08057974106C042E09D
:1007B00061E080E797E1821B930B0E947C018091AE
:1007C00031049091320426E1883A920758F48091DE
:1007D00004048337B0F081508093040480910504B1
:1007E00081500DC08953984178F0809104048F376F
:1007F00040F48F5F80930404809105048F5F8093A1
:10080000050410924204BFC117E71093040410932B
:100810000504809142048F5F80934204853009F083
:10082000B2C180E00E94D30784E693E00E943B08B7
:1008300010930404109305048091310490913204C4
:10084000909334048093330482E380932E041092B7
:10085000420486C18CE880930304209137043091D0
:1008600038048091390490913A048217930798F4E0
:1008700080E00E94D30785E793E00E943B0888E66A
:100880008093040486E88093050483E48093030442
:1008900010923F0413C080E00E94D30784E893E0E5
:1008A0000E943B0886E88093040488E68093050450
:1008B00080ED8093030481E080933F0482E319C0BC
:1008C00087E780930404809305048AE080932E04D4
:1008D00082E08093400418C080E00E94D30780E249
:1008E00093E00E943B0886E880930404809305040B
:1008F00084E180932E0434C18FE7809304048093B5
:1009000005048AE080932E0481E13BC10E948C0B98
:1009100083E080932E040E94A70B882309F433C13F
:100920000E94A00B909332048093310481E0E1CFC8
:10093000809141048F5F8093410490914004891716
:1009400048F083E180932F0481E080932E0410927D
:10095000410419C180913F04882309F047C00E94D7
:10096000D30783E993E00E943B0820913104309142
:10097000320487E12137380730F042E063E0C901F3
:100980008057974106C042E062E080E797E1821B12
:10099000930B0E947C01609131047091320480912C
:1009A0003504909136046817790770F423E16838AC
:1009B000720728F488E68093040486E84AC06656E5
:1009C000774108F07CC073C08617970708F077C09E
:1009D0008BE16935780728F086E88093040488E67F
:1009E0004EC06B57774108F46AC039C0813009F0B6
:1009F0006EC080E00E94D30784EA93E00E943B0827
:100A0000209131043091320447E12137340730F02E
:100A100042E062E0C9018057974106C042E063E0CE
:100A200080E797E1821B930B0E947C016091310467
:100A300070913204809135049091360468177907DB
:100A400098F483E16838780738F486E880930404E2
:100A500088E68093050426C06656774180F586E8CF
:100A60008093040488E627C08617970740F54BE17A
:100A700069357407C8F088E68093040486E880939B
:100A8000050480E090E0605777418040904028E284
:100A900030E040E050E00E94E70B2F3018F4209344
:100AA0002E0415C08FE011C06B57774140F088E6E7
:100AB0008093040486E88093050485E006C08FE7F0
:100AC000809304048093050484E080932E04809135
:100AD00031049091320490933604809335048091D0
:100AE0002F0482504EC08CE88093030487E78093E4
:100AF00004048093050483E280932E0484E141C0C2
:100B000083E080932E040E948C0B0E94A70B882305
:100B1000D1F10E94A00B909332048093310427E11D
:100B20008037920740F441E060E080E090E00E946E
:100B30007C0182E026C09C0120573741805E9E42A6
:100B400038F441E060E0C9010E947C0182E006C007
:100B500041E060E0C9010E947C018AE0809340048A
:100B600080912F048F5F0DC080913F04882311F482
:100B700083E401C080ED8093030485E080932E041C
:100B80008FE080932F0410922D0420913B0422309B
:100B900009F001C180912D048F5F80932D04909105
:100BA0002E04891708F4F7C080912F04843009F4CB
:100BB00068C0853050F4813011F18130C8F0823046
:100BC00059F1833009F0E5C04EC0873009F47CC08C
:100BD000883038F4853009F45DC0863009F0D9C01A
:100BE00061C0883009F478C0893009F0D2C0C6C02D
:100BF0000E94DF0781E00E94A80781E0B9C080E081
:100C00000E94D30780E293E00E943B0886E880932D
:100C100004048093050456C08FE7809304048093F6
:100C200005040E948C0B83E080932E040E94A70B86
:100C3000882309F4AEC00E94A00B909332048093E5
:100C4000310425E18C37920738F442E060E080E01F
:100C500090E00E947C018EC042E060E08C5795419C
:100C60000E947C0196C080E00E94D30781E393E05C
:100C70000E943B088CE6809304048093050482E381
:100C800077C087E7809304048093050420932E04A3
:100C900085E07DC08EEA8093030484E180932E0476
:100CA00086E075C00E948C0B84E080932E040E9425
:100CB000A70B882309F46DC00E94A00B9093380401
:100CC0008093370484E154C087E68093030488E26C
:100CD00080932E0488E05BC00E948C0B84E080939C
:100CE0002E040E94A70B882309F453C00E94A00B76
:100CF0009C0190933A04809339048CE88093030418
:100D0000809137049091380445E18C37940798F42A
:100D100045E12C37340778F480E00E94D30785EB57
:100D200093E00E943B0888E68093040486E8809361
:100D3000050486E41DC02817390760F480E00E948E
:100D4000D30786EC93E00E943B0888E68093040476
:100D500086E80BC080E00E94D30787ED93E00E94F5
:100D60003B0886E88093040488E68093050488E2C3
:100D700080932E0480912F048F5F09C087E78093B2
:100D80000404809305048AE080932E0481E080931C
:100D90002F0410922D0480913B04833009F046C04B
:100DA00080912D048F5F80932D0490912E048917DC
:100DB000E8F180912F04882319F08130A9F51CC037
:100DC0000E94DF0781E00E94A80780E00E94D3070D
:100DD00088EE93E00E943B0880E10E94D30788EFF1
:100DE00093E00E943B0881E080932E0480912F04C1
:100DF0008F5F80932F0418C00E948C0B8AE0809331
:100E00002E040E94A70B882379F00E94A00B9093D8
:100E10003204809331048AE10E94D3078091310427
:100E2000909132040E94800810922D041F91089521
:100E3000CF93DF93F8940E94E8000E9440090E943B
:100E4000B0090E94300A0E94AB0B82E30E9499070E
:100E500082E00E94A8078CE990E00E942D080E9481
:100E6000BB090E94420A7894C0E6D1E08091300428
:100E7000882321F0109230040E949B02CC9908C074
:100E800080913D04882359F183E00E945B0125C0D5
:100E9000CD9B10C0CC9B0EC080913D048823F9F4FB
:100EA0000E946F0110923C0481E080933D040E94F7
:100EB000180715C0CD9913C080913D04882379F09F
:100EC00080E00E94A807CE010E942D0881E0809357
:100ED0003C040E94BF090E94450A10923D04CE992D
:100EE00006C080913E04882309F281E01BC0CF9B9D
:100EF00011C0CE9B0FC080913E04882309F0B6CF6D
:100F00000E946F0110923C0481E080933E040E9495
:100F10001807ACCFCF99AACF80913E04882309F45B
:100F2000A5CF82E00E945B0110923E049FCF9927DB
:100F3000089581BF08951F93182F0E94F90A80E039
:100F40000E94FC0AC198812F0E94EF0A1F91089508
:100F5000813051F0813018F08230F9F412C089E309
:100F60000E949B078DE10AC089E30E949B078CE1E8
:100F70000E949B078EE30E949B0780E10E949B07D3
:100F8000089589E30E949B078CE10E949B078EE3F2
:100F90000E949B0788E10E949B0708958F708067DD
:100FA0000E949B07089580680E949B07089582E035
:100FB0000E949B0780E49FE10197F1F7089581E08B
:100FC0000E949B0780E49FE10197F1F70895882331
:100FD00031F0813049F480914304816003C08091F5
:100FE00043048E7F809343048091430488600E9471
:100FF0009B070895882331F0813049F480914304A0
:10100000826003C0809143048D7F8093430480916C
:10101000430488600E949B070895882331F0813043
:1010200049F480914304846003C0809143048B7F22
:10103000809343048091430488600E949B07089535
:101040001F93182F0E94F90A80E00E94FC0AC19A9F
:10105000812F0E94EF0A1F910895CF93DF93EC0137
:1010600002C00E942008FE01219684918823C9F7BE
:10107000DF91CF910895CF93DF93EC0102C00E94DE
:10108000200889918823D9F7DF91CF910895CF93D4
:10109000DF93CDB7DEB727970FB6F894DEBF0FBE4C
:1010A000CDBFBC0180E3898388E78A83FE01339644
:1010B0004CE050E033E0CB01042E02C096958795BA
:1010C0000A94E2F7282F2F708F7090700A9710F013
:1010D000295C01C020632083445050403F5F31961B
:1010E000373049F71F82CE0101960E943B082796B0
:1010F0000FB6F894DEBF0FBECDBFDF91CF9108953C
:101100008F929F92AF92BF92CF92DF92EF92FF9217
:101110000F931F93CF93DF93CDB7DEB725970FB60D
:10112000F894DEBF0FBECDBF8C01DE011196E8E062
:10113000F4E085E001900D928150E1F7C80160E193
:1011400077E20E94D30BFB01E62E262F332780E1A6
:1011500097E2289F6001299FD00C389FD00C112462
:10116000C8018C199D0968EE73E00E94D30BF62E1E
:10117000262F332788EE93E0289F4001299F900C6B
:10118000389F900C112494012C0D3D1DC801821B29
:10119000930B64E670E00E94D30B462F84E6689FB1
:1011A000500111242A0D3B1DC801821B930B6AE0DC
:1011B00070E00E94D30BEE2311F430E004C08E2FB8
:1011C0008063898331E0FF2011F4EE2039F0FE01C5
:1011D000E30FF11D8F2D806381833F5F442321F452
:1011E000FF2011F4EE2039F0FE01E30FF11D842FF2
:1011F000806381833F5F662331F4442321F4FF2021
:1012000011F4EE2039F0FE01E30FF11D862F80630B
:1012100081833F5FAE014F5F5F4FFA01E30FF11D26
:10122000202F2C1928192A198AE0689FC00111243F
:10123000281B20632083232F04C0AE0FBF1F80E232
:101240008C932F5FDA01E22FFF272530B0F3E40FF4
:10125000F51F1082CA010E943B0825960FB6F8942C
:10126000DEBF0FBECDBFDF91CF911F910F91FF90D9
:10127000EF90DF90CF90BF90AF909F908F900895A8
:101280000E94060B87B3836087BB83B78A6683BFE0
:1012900080E00E94A80780E50E949B078CE60E94E0
:1012A0009B0786E00E949B0781E00E940D0880E07A
:1012B0000E94FA0780E00E94E70786E00E94CE07BE
:1012C0000E94DF0711BE08951092450486E494E061
:1012D00008951092440495980895809145049927A3
:1012E00008951F920F920FB60F9211242F933F93E0
:1012F0004F935F936F937F938F939F93AF93BF931E
:10130000EF93FF930E94300B90914404992331F4A2
:101310008A30A9F481E08093440411C09B3048F4E2
:10132000E92FFF27EB5BFB4F80839F5F9093440483
:1013300006C09B3021F4959A81E080934504FF918B
:10134000EF91BF91AF919F918F917F916F915F913D
:101350004F913F912F910F900FBE0F901F901895B6
:101360000E943D0B80E699E00E94100B109244040D
:101370008D9A959808950E943B0B959A089595989B
:101380000E94390B089580910E0410920E04992743
:101390000895BC0140E050E020E030E0FB01E20FA6
:1013A000F31F8081480F511D2F5F3F4F2C303105B7
:1013B000A9F7842F992708951F931091620486E559
:1013C00094E00E94C909181751F580915704992794
:1013D0008F709070892B19F5809158048234B1F088
:1013E000833428F4803261F08134C9F40CC0843431
:1013F00099F0843470F08A3F91F485E090E011C058
:1014000081E090E00EC082E090E00BC083E090E0CD
:1014100008C084E090E005C086E090E002C080E073
:1014200090E01F910895DC01E1E1F4E08D9181935A
:1014300084E0EB31F807D1F7CF010C970E94C9097E
:1014400080931B0481E08093540408958091530499
:10145000992708951092520481E0809355040895CD
:101460000E947D0B80E895E20E944C0B8C9A1092B2
:10147000520481E0809355041092540484E08093D8
:101480000E0408950E94790B08950E94750B08952B
:10149000CF93DF93949A80E49CE9FC013197F1F7B4
:1014A000FC013197F1F7FC013197F1F70197F1F762
:1014B00080E00E94710B80E00E94710B80E00E942E
:1014C000710B80915404882351F0CFE0D4E08991CE
:1014D0000E94710B84E0CC31D80751F0F8CFCCE1F9
:1014E000D4E089910E94710B84E0C932D807C9F712
:1014F00080E00E94710B80E00E94710B80E00E94EE
:10150000710B949880E89EE30197F1F7DF91CF91FA
:1015100008951F920F920FB60F9211242F933F93AD
:101520004F935F936F937F938F939F93AF93BF93EB
:10153000EF93FF930E946C0B90915204992341F416
:101540008A3081F48093560481E0809352040AC06B
:101550009D3040F4E92FFF27EA5AFB4F80839F5FBD
:1015600090935204809152048D3041F50E94420ABA
:1015700078940E94DC09809353048330A1F0843076
:1015800028F4813051F08230A9F40DC0853071F01B
:10159000853040F0863071F406C080930E040E94BE
:1015A000480A08C084E080930E0404C080930E04AF
:1015B00010925404109252040E94450AFF91EF9138
:1015C000BF91AF919F918F917F916F915F914F915B
:1015D0003F912F910F900FBE0F901F9018958FB9CC
:1015E000779BFECF08958FB19927089568986998E1
:1015F00008956898699A089521E030E002C0220FAA
:10160000331F8A95E2F720952BBB089587B3806B33
:1016100087BBC69AD09AD89A8DB181658DB9089545
:101620009C0194E0220F331F9A95E1F74427552738
:1016300060E074E284EF90E00E94090C2150304099
:1016400040405040BB2757FDBA95A52F942F832FBC
:101650002F5F3F4F4F4F5F4F80BD215029B90895F5
:101660005F9BFECF8CB1992708955D9BFECF8CB90F
:101670000895579A089557980895899A8AB1886964
:101680008AB90895FC0104C05D9BFECF8CB93196E8
:1016900080818823C9F708959C0194E0220F331FAD
:1016A0009A95E1F74427552760E074E284EF90E0D3
:1016B0000E94090C2150304040405040BB2757FD4C
:1016C000BA95A52F942F832F2F5F3F4F4F4F5F4F1A
:1016D0008CBF215020B90895179BFECF83B1992765
:1016E0000895159BFECF83B9089581B1806981B9B2
:1016F000089581B18F7681B90895BB9A81B18869C7
:1017000081B90895FC0104C0159BFECF83B93196C1
:1017100080818823C9F70895F89480916404882310
:1017200069F48A9A929A8AE08A95F1F792988A984F
:1017300085B7836085BF8BB780648BBF789408952D
:10174000109264048091880090918900089580919E
:1017500064049927089508951F920F920FB60F926F
:1017600011248F9305B600FE0DC0109289001092CF
:10177000880085B78E7F85BF80918A0082608093C4
:101780008A000BC080918A008D7F80938A0081E05F
:10179000809364048BB78F7B8BBF8F910F900FBEAC
:1017A0000F901F901895AA1BBB1B51E107C0AA1FE1
:1017B000BB1FA617B70710F0A61BB70B881F991FF2
:1017C0005A95A9F780959095BC01CD010895A1E2A5
:1017D0001A2EAA1BBB1BFD010DC0AA1FBB1FEE1FAB
:1017E000FF1FA217B307E407F50720F0A21BB30BF6
:1017F000E40BF50B661F771F881F991F1A9469F772
:1018000060957095809590959B01AC01BD01CF01CD
:10181000089597FB092E05260ED057FD04D0D7DF7B
:101820000AD0001C38F450954095309521953F4FD3
:101830004F4F5F4F0895F6F790958095709561959D
:0A1840007F4F8F4F9F4F0895FFCF99
:10184A00202020202020202020202020202020208E
:10185A00003E202020202020202020202020202080
:10186A003C003E3E20202020202020202020202036
:10187A003C3C003E3E3E20202020202020202020EC
:10188A003C3C3C003E3E3E3E2020202020202020A2
:10189A003C3C3C3C003E3E3E3E3E20202020202058
:1018AA003C3C3C3C3C003E3E3E3E3E3E202020200E
:1018BA003C3C3C3C3C3C003E3E3E3E3E3E3E2020C4
:1018CA003C3C3C3C3C3C3C003E3E3E3E3E3E3E5B5D
:1018DA005D3C3C3C3C3C3C3C002020202020203C01
:1018EA0020203E2020202020200020202020203CD4
:1018FA003C20203E3E202020202000202020203C8A
:10190A003C3C20203E3E3E20202020002020203C3F
:10191A003C3C3C20203E3E3E3E2020200020203CF5
:10192A003C3C3C3C20203E3E3E3E3E202000203CAB
:10193A003C3C3C3C3C20203E3E3E3E3E3E20003C61
:10194A003C3C3C3C3C3C20203E3E3E3E3E3E3E0033
:10195A003C3C3C3C3C3C3C5B5D3E3E3E3E3E3E3E6F
:10196A00003C3C3C3C3C3C3C2020202020202020C9
:10197A002000203C3C3C3C3C3C20202020202020D5
:10198A0020200020203C3C3C3C3C202020202020E1
:10199A00202020002020203C3C3C3C2020202020ED
:1019AA002020202000202020203C3C3C20202020F9
:1019BA0020202020200020202020203C3C20202005
:1019CA00202020202020002020202020203C202011
:1019DA002020202020202000202020202020205BE2
:1019EA005D202020202020200020202020202020D0
:1019FA0020203E3E3E3E3E3E3E002020202020202B
:101A0A002020203E3E3E3E3E3E2000202020202038
:101A1A00202020203E3E3E3E3E2020002020202046
:101A2A0020202020203E3E3E3E2020200020202054
:101A3A002020202020203E3E3E2020202000202062
:101A4A00202020202020203E3E2020202020002070
:101A5A0020202020202020203E202020202020007E
:101A6A0044726976653A20464F52574152442020C3
:101A7A000044726976653A2053544F502020202042
:101A8A002000416C69676E20746F2077616C6C204E
:101A9A0020200020205E2D2D2028316D29202D2D7B
:101AAA005E202000506F73697374696F6E206C6FCB
:101ABA00636B65640044726976653A205475726E88
:101ACA00203C200044726976653A205475726E2073
:101ADA003E2000205D2D2D2D2028316D29202D2D11
:101AEA002D3E7C007C3C2D2D2D2028316D29202D6A
:101AFA002D2D5B200044726976653A205475726E0A
:101B0A00203C3C3C200044726976653A2054757248
:101B1A006E203C2020200044726976653A20547574
:101B2A00726E203E20202000536572766F3A20663E
:101B3A006F7277617264200044697374616E6365C1
:101B4A003A20008C77777777202020202000040A1B
:101B5A004030000000000000000000000A803055FC
:0A1B6A005555555555555555B70012
:00000001FF
